:1000000009C016C015C014C013C012C011C010C062
:100010000FC00EC011241FBECFE9CDBF20E0A0E667
:10002000B0E001C01D92A136B207E1F766D0B0C0C2
:10003000E7CF88B3826188BB089588B3826188BBAB
:100040008FE295E70197F1F700C0000088B38D7E3D
:1000500088BB9FE320E982E0915020408040E1F797
:1000600000C00000089588B3826188BB8FE295E7E5
:100070000197F1F700C0000088B38D7E88BB8FE246
:1000800095E70197F1F700C0000088B3826188BB53
:100090008FE295E70197F1F700C0000088B38D7EED
:1000A00088BB9FE320E982E0915020408040E1F747
:1000B00000C000000895C19AC4982FEB84ED91E030
:1000C000215080409040E1F700C00000C49AC198E0
:1000D0002FEB84ED91E0215080409040E1F700C08B
:1000E00000000895C29A87B3847087BB88B38D7E61
:1000F00088BB87B3826187BB0895F4DF10926000EC
:10010000B299FECFB29BFECF87E691E00197F1F75F
:1001100000C00000B29B05C0809160008F5F80939B
:10012000600090E59A95F1F70000B29B05C08091C0
:1001300060008F5F8093600080E58A95F1F7000092
:10014000B29B05C0809160008F5F8093600090E556
:100150009A95F1F70000B29B05C0809160008F5F17
:100160008093600080916000811101C062DF809106
:100170006000813009F461DF80916000823009F411
:1001800072DF80916000833009F0B8CF94DFB6CF82
:04019000F894FFCF11
:00000001FF
